:10000000008000205D030000A5030000A70300009E
:10001000A9030000AB030000AD03000000000000D6
:10002000000000000000000000000000AF0300001E
:10003000B103000000000000B3030000B50300009E
:10004000B7030000B7030000B7030000B7030000C8
:10005000B7030000B7030000B7030000B7030000B8
:10006000B7030000B7030000B7030000B7030000A8
:10007000B7030000B7030000B7030000B703000098
:10008000B7030000B7030000B7030000B703000088
:10009000B7030000B7030000B7030000B703000078
:1000A000B7030000B7030000B7030000B703000068
:1000B000B7030000B70300000000000000000000CC
:1000C000B7030000B7030000B7030000B703000048
:1000D000B7030000B7030000B7030000B703000038
:1000E000B703000000000000000000000000000056
:1000F00000000000B703000000000000B70300008C
:1001000000000000000000000000000000000000EF
:1001100000000000000000000000000000000000DF
:1001200000000000000000000000000000000000CF
:1001300000000000000000000000000000000000BF
:1001400000000000000000000000000000000000AF
:10015000000000000000000000000000000000009F
:10016000000000000000000000000000000000008F
:10017000000000000000000000000000000000007F
:10018000000000000000000000000000000000006F
:10019000000000000000000000000000000000005F
:1001A000000000000000000000000000000000004F
:1001B000000000000000000000000000000000003F
:1001C000000000000000000000000000000000002F
:1001D000000000000000000000000000000000001F
:1001E000000000000000000000000000000000000F
:1001F00000000000000000000000000000000000FF
:10020000354936480A1A02D0072291438D463449AF
:1002100034480A1A06D00722914381F30988022242
:1002200082F3148830483149314A00F044F83148AB
:100230003149324A00F03FF831483249324A00F041
:100240003AF832483249334A00F035F832483349F7
:10025000334A00F030F833483349344A00F02BF881
:1002600033483449344A00F026F8344834490022EF
:1002700000F02CF833483449002200F027F83348C6
:100280003349091A082902DB002202604160314A21
:1002900090471F481F49884205D00268043003B4C4
:1002A000904703BCF7E700208646EC46002000217B
:1002B000294A9047FEE7884207D0521A05D00378B2
:1002C00001300B700131013AF9D17047884202D0F8
:1002D00002700130FAE770470080002000700020B3
:1002E0000080002000800020480500000000002061
:1002F00004000020BC030000BC0300003405000023
:100300004805000000000020000000203405000027
:1003100034050000340500003405000034050000F9
:1003200034050000340500003405000046050000D7
:100330004C05000004000020040000200400002000
:10034000040000200400002004000020040000201D
:100350000410002073030000BD03000000F02CB85F
:100360000B484FF00701884385460A488047FFF74E
:1003700047BF094809490A4A884207D0521A05D09E
:10038000037801300B700131013AF9D17047000058
:1003900000800020E503000034050000000000207C
:1003A00000000020FEE7FEE7FEE7FEE7FEE7FEE7CF
:0C03B000FEE7FEE7FEE7FEE7FFF7D2BF26
:1003BC0008B5084D42F2107445F001054FF47A402F
:1003CC00A847013CFAD14FF080430122C3F8002525
:1003DC00FEE700BF400500004C4B1B680D2B57D1AE
:1003EC004FF080414FF080520023C1F80C31C1F81E
:1003FC001031C1F83835464BD2F80404C3F8200547
:10040C00D2F80804C3F82405D2F80C04C3F8280564
:10041C00D2F81004C3F82C05D2F81404C3F8300534
:10042C00D2F81804C3F83405D2F81C04C3F84005FC
:10043C00D2F82004C3F84405D2F82404C3F84805C4
:10044C00D2F82804C3F84C05D2F82C04C3F8500594
:10045C00D2F83004C3F85405D2F83404C3F860055C
:10046C00D2F83804C3F86405D2F83C04C3F8680524
:10047C00D2F84004C3F86C05D2F84424C3F87025B4
:10048C00D1F80034DB0744BF6FF00103C1F800342E
:10049C004FF01023D3F80022002A03DBD3F80432E8
:1004AC00002B2FDA1B4B0122C3F80425D3F80024B0
:1004BC00002AFBD04FF010221221C2F80012D3F800
:1004CC000024002AFBD04FF010231222C3F8042280
:1004DC00104B1A46D3F800140029FBD00021C3F8A6
:1004EC000415D2F80034002BFBD0BFF34F8F0A4910
:1004FC000A4BCA6802F4E0621343CB60BFF34F8F20
:10050C0000BFFDE7064B074A1A6070473001001028
:10051C0000C0004000E0014000ED00E00400FA05DE
:08052C00000000200090D00344
:100534000000000000000000000000000338FDD8A7
:020544007047FE
:040548000090D0034C
:040000030000035D99
:00000001FF
